:030000000211D119
:03000B000200BE32
:03002B000203E0ED
:03005B0002052477
:0300730002051A69
:1000800002030406080C10182030406080020304AC
:1000900006080C101820304080FF0406080C1018C9
:1000A0002030406080A0C000000001010003020277
:1000B000010505020D0505050D0603050202C2AF87
:1000C000C0D0C0E0205A25302F02E47330601A05FA
:1000D00060C37405952540F2956040EE758A78E519
:1000E000257003758A000203D90203CC306306C26F
:1000F00095C294C29385258AC25AE525F4700221DF
:10010000BF0561306013206A19758B00D0E0D0D034
:10011000C295C294C293D2AF32C295C294C2930226
:1001200001AFD26EC26FE565601CC3E561149565D1
:100130004014C26ED26FC3E561956450030201AFF3
:100140007561000201AF206C14C295C294C2937411
:1001500001D5E0FDC292C291C2900201AFC295C228
:1001600094C293E53D20E22520E10D207502C29264
:10017000307502C2900201AF20E005C2910201AFCA
:10018000207502C290307502C2920201AF20E115C3
:1001900020E00D207502C292307502C2900201AFBC
:1001A000C2910201AF207502C290307502C29275F1
:1001B0008B00D0E0D0D0C295C294C293D2AF32D0DF
:1001C000E0D0D0D2AF3261CCE525600A207502D2F2
:1001D00095307502D293C29461CCE5256002D29429
:1001E000207502C293307502C29561CCE525600A84
:1001F000207502D293307502D295207502C29530D7
:100200007502C29361CC207502D292307502D290F1
:10021000E525600A207502D295307502D2932075CB
:1002200002D290307502D292C29461CC207502D273
:1002300092307502D290207502D290307502D2921F
:100240007401D5E0FDE525600A207502D295307570
:1002500002D293C29461CC207502D292307502D240
:1002600090E525600A207502D295307502D293D2AE
:1002700091C29461CC207502D292307502D290D294
:10028000917401D5E0FDE525600A207502D2953014
:100290007502D293C29461CCD291E5256002D294CA
:1002A000207502D292307502D290207502C293302E
:1002B0007502C29561CCD291207502D2923075023E
:1002C000D2907401D5E0FDE5256002D2942075023C
:1002D000C293307502C29561CCD291E5256002D2FD
:1002E00094207502D290307502D292207502C2938A
:1002F000307502C29561CCD291207502D2903075D2
:1003000002D2927401D5E0FDE5256002D2942075F9
:1003100002C293307502C29561CC207502D2903032
:100320007502D292E525600A207502D293307502DB
:10033000D295D291207502C295307502C29361CCDC
:10034000207502D290307502D292D2917401D5E01C
:10035000FDE525600A207502D293307502D2952002
:100360007502C295307502C29361CC207502D2909D
:10037000307502D292E525600A207502D29330755D
:1003800002D295207502D292307502D29020750269
:10039000C295307502C29361CC207502D29030753F
:1003A00002D292207502D292307502D2907401D599
:1003B000E0FDE525600A207502D293307502D295E2
:1003C000207502C295307502C29361CCE525F4F523
:1003D0008A758B00756000D25AD0E0D0D0D2AF328F
:1003E000C2AFC0D0C0E0D2D3C2CEE528600A741F2D
:1003F000552E60491528813D78007900E5803076DA
:1004000001F430E70278FF53DACF20760343DA2095
:1004100030760343DA10C2D8C269E580307601F441
:1004200030E70279FFC3E89970CE30590375281878
:10043000741F552E60037528188858D268E5296006
:100440000415298150741F552E600543DA01C2D866
:1004500020680281E2E558F8C268741F552E6036A4
:100460007982B70431C3E894F0400374F0F8E8C42B
:0F047000540F28F87984B703028196C313C3137E
:10047F008721200802C313200A06C3C898F8819663
:10048F0028F8500374FFF8C3E8955F5003E55FF851
:10049F00E52C5406703D882230630AC3E522955C33
:1004AF004003855C227882B60429C3E52295244057
:1004BF001278A096400DE52426F52450097524FFE7
:1004CF000204D5852224852425C3E524955C4003A9
:1004DF00855C2520CF09D0E0D0D0C2D3D2AF32C2B5
:1004EF00CF7801E5286008741F552E70021528C3B8
:1004FF00E55894014005755B00A111E55B046002AE
:10050F00055BD0E0D0D0C2D3D2AF32C2AF53917F10
:10051F00C258D2AF32C2AFC0D0C0E0C0F0D2D3A861
:10052F00FBA9FCC2D8306902A18753DACF2076032A
:10053F0043DA1030760343DA20D269E58030760152
:10054F00F420E702A15B88268927E12753DACF2021
:10055F00760343DA2030760343DA10C2D8C26974C7
:10056F001F552E7002E10D7800E580307601F430D2
:10057F00E702E10D8858E10D53DACF20760343DA15
:10058F002030760343DA10C269205902C14153DA91
:10059F00CF20760343DA1030760343DA20C2D8D265
:1005AF006988538954C3E89551F8E99552F9E4FBEA
:1005BF007AFAC3E894C8E994005008E4D2E4FB7ACD
:1005CF000AC114C3E89468E994015008E4D2E3FB2C
:1005DF007A0FC114C3E894D0E994025008E4D2E230
:1005EF00FB7A1EC114C3E894A0E994055008E4D225
:1005FF00E1FB7A3CC114C3E89498E994085006E4EF
:10060F00D2E0FB7A78C3E89555FCE99556FD30E7C3
:10061F0008ECF42401FCEDF4FD7557007008C3ECF1
:10062F009A500375570188558956A853A954885174
:10063F008952C3E89526F8E99527F9307402C1E08D
:10064F00307302C1E0307202C1D9E9C313F9E81364
:10065F00F8307102C1D9E9C313F9E813F830700209
:10066F00C1D9E9C313FDE813FC205918C3EC941C3E
:10067F00ED9402400302070DED7009C3EC94C850CE
:10068F000302072774002077037896E624FAFEE426
:10069F003400FFC3EC9EFCED9FFD500678007900FF
:1006AF00C1E0C3EC94FFED9400400678FF7900C1E0
:1006BF00E0EC856CF0A4C5F0A2F733F879004003A5
:1006CF000206FC78FF79000206FCE9C313F9E81370
:1006DF00F830740EE9600278FFC3E81338F8E43499
:1006EF0000F9C3E894FFE99400400278FF8858D2DC
:1006FF0068205902E10D741FF4552E4BF52E752805
:10070F0018741F552E700375280A305902E127748B
:10071F001F552E600353DAFE752906741F552E7070
:10072F000375290AD0F0D0E0D0D0C2D3D2AF32793E
:10073F0001E1567903E156790AE156791EE15679BE
:10074F0064E15679C8E1567817E4D5E0FDD8FAD9B7
:10075F00F6227A147B7802077D7A107B8C02077D54
:10076F007A0D7BB402077D7A0B7BC802077DAC251F
:10077F007525017902B275E4D291D5E0FDE52560CA
:10078F0002D294D5E0FDC294D5E0FDC291D5E0FD33
:10079F00E525600A207502D295307502D293E56D7A
:1007AF00D5E0FD207502C295307502C2937496D5BF
:1007BF00E0FDD9C1EAF8D5E0FDD8FBDBB1D2918CD1
:1007CF002522C37C007D0075F00005F0EA33FAEBBB
:1007DF0033FB50F6EB13FBEA13FAC3E9FFE8FEE82D
:1007EF009AF8E99BF95004EFF9EEF8B3EC33FCED0E
:1007FF0033FDD5F0DFEDF9ECF822E889F08A20D24D
:10080F00D4F8A9F07B0030F70B7BFFF42401F8E953
:10081F00F43400F9E88520F0A4ADF0F8E98520F074
:10082F00A4AFF0FEED2EF974003FFA7C04C3EA1377
:10083F00FAE913F9E813F8DCF48BF030F70AE8F46F
:10084F002401F8E9F43400F9E889F0C2D4F8A9F0EA
:10085F00227882B604030208ECC3E55894014018CD
:0F086F00E54870377805C37994B702027812C351
:10087E00E53B9400E53C984020E5486009855E5DC7
:10088E007562FF756301852224E4F53FF540F5415D
:10089E00F542F543F5480208EC754801C37994E733
:1008AE009402601BE523F43333F913F8E954010481
:1008BE00F9E854FEC39440F8E99400F90208E8E51B
:1008CE0023F433333333F913F8E954070404F9E806
:1008DE0054F8C39440F8E99400F9883F894022E522
:1008EE0048603BC3E53C13F9E53B13F8C3E53F987D
:1008FE00F8E54099F9500CC3E89480E994FF40164E
:10090E00020928C3E8947FE994005003020928786D
:10091E007F7900020928788079FF8844894522E58D
:10092E00486058E5442541F8E5453542F9854520AE
:10093E00E4300701F43543FA30E709C3EA94F04096
:10094E001502096AC3EA940F500302096A78FF7907
:10095E00FF7A0F02096A780079007AF0C3E52495D0
:10096E005C5006E52460092183E54520E70D2183CF
:10097E00E54530E706884189428A4322E5487003FF
:10098E000209ED789EE6FAC3E54433F8E54533F9FE
:10099E001109E930E70BC3E89480E994FF40132175
:1009AE00C4C3E8947FE99400500221C4787F790093
:1009BE0021C4788079FFE820E715C3E52398F84035
:1009CE0009C3E8940140030209EB78010209EBE840
:1009DE00F424012523F840030209EB78FF88462210
:1009EE00E5487003020A4F789FE6FAA842A9431120
:1009FE0009E930E70CC3E89401E994FF4016020AB6
:100A0E0026C3E894FFE994005003020A2678FF7982
:100A1E0000020A26780179FFE920E715C3E546981A
:100A2E00F84009C3E894014003020A4D7800020A17
:100A3E004DE8F424012546F84003020A4D78FF885C
:100A4E002422020AE77883E6F520120F4A75E89011
:100A5E00E5E820ECEDA8BDA9BE120FE2756855754C
:100A6E006900C3740013FD745513FC74552CFC748B
:100A7E00003DFDECFAEDFBC3E89AE99B4014E568F6
:100A8E002455F568E5693400F569EA2CFAEB3DFB6F
:100A9E0080E5AE68AF69C3E56913F9E56813F8C37D
:100AAE00E913F9E813F8E56828F566E56939F5679D
:100ABE007A03C3E913F9E813F8DAF7AA201A7009D2
:100ACE00756800756900020AE71AEA6008EE28FEEA
:100ADE00EF39FFDAF88E688F692275E890227883F5
:100AEE00E6FFE5E820ECF7A8BDA9BE056AC3E56AF6
:100AFE0094084052756A00E97007E56B601B020BA3
:100B0E001BC3E8956B6010E56B5006600C14020B6E
:100B1E00270460F9020B27E56BF56BC3946DF84063
:100B2E0021755CC0C3E89404F84017755C80C3E877
:100B3E009404F8400D755C40C3E89404F8400375C6
:100B4E005C0075BB0622C3E56AB4070375BB1022B1
:100B5E0030610278323062027878E52C5406601FDC
:100B6E00E879A187F0A4C5F0A2F733F8C3E8955C45
:100B7E004002A85C882288248825306102885E2283
:100B8E00788FE6FFC3EF94055018C3EF94045020FE
:100B9E00C3EF94035028C3EF94025030C3EF940177
:100BAE0050387533A075340F75353C75360561F6C2
:100BBE007533C075341275354075360661F675336A
:100BCE00707534177535D075360761F675334C75FB
:100BDE00341D7535C475360961F6753328753423A1
:100BEE007535B875360B61F685334F853450753BC8
:100BFE0000753C0822A84FA950020C0EA849A94A1C
:100C0E00759100C3E498F594E499F595759104D225
:100C1E005875C820A8CCA9CD75C824AA39AB3A8876
:100C2E0039893AC3E89AF8E99BF9AA3BAB3CC3EB86
:100C3E0013FDEA13FCC3ED13FDEC13FCC3EA9CFA9F
:100C4E00EB9DFBEA28FAEB39FB8A3B8B3C400122F9
:100C5E00753BFF753CFF223058028165759100C3CC
:0F0C6E00E4954BF594E4954CF595759104D258A7
:100C7D00227892E6FF7E10305B027F053063047FA1
:100C8D00037E00A93CA83B7A04C3E913F9E813F8E5
:100C9D00DAF7C3E89EF8E99400F94009C3E8940235
:100CAD00E9940050047802E4F9E9FBE8FAC3E9138A
:100CBD00FDE813FCC3EF9403602EEF20E00DE82C4C
:100CCD00F8E93DF9ECFAEDFB020CE2E828F8E93918
:100CDD00F97A02E4FBC3EF9403400D8A4D8B4E88E5
:100CED0049894A8C4B8D4C22884D894E8A498B4AB5
:100CFD008C4B8D4C22305802A102759100C3E495A6
:100D0D003BF594E4953CF595759104D25822753ECA
:100D1D0000752000020D2A753E00752040D2AF05EA
:100D2D003E20580122759D00E53CC313C313F808FE
:100D3D006030306A06C313C313F808C3E8940A4041
:100D4D0002780A306D08C3E8940440027804C3E5C4
:100D5D003C9408400D759D02C3E53C94104003750D
:100D6D009D03205803D2AF22790F206D027905D251
:100D7D00AF0000C2AF205A0A7914206D02790730F6
:100D8D006FE03063027978C3E58B9940D5E59BF42C
:100D9D005440B52002A12AD8C9D2AF22C25B789C9B
:100DAD00E6146007E53E147002D25B30630B053824
:100DBD00205810753800020DD02058071581158167
:100DCD0002172322759100C3E4954DF594E4954ED9
:100DDD00F595759104D25822AE25305B4F78A3E678
:100DED00FFBF010BD25C752500C295C294C29391D1
:100DFD006A305C03752500305802A1FEBF020BD28C
:100E0D005C752500C295C294C29378A2B6010D916E
:100E1D006A305C03752500305802C11EBF030BD22A
:100E2D005C752500C295C294C293B1D1305C037537
:100E3D002500305802C139305B04C25C8E2522C2B8
:100E4D00AFD291206A03020E6E90031A206C1230FD
:100E5D006E0F207502D290307502D2927401D5E0DA
:100E6D00FD207502C292307502C290759F11753DBD
:100E7D0002D2AF22C2AF206A03020EA39002D93074
:100E8D006E17D291207502D290307502D2927401F4
:100E9D00D5E0FD020EA69001DA207502C2933075E1
:100EAD0002C295305A06E5256002D294207503756D
:100EBD009F01307503759F21753D03D2AF22C2AFDF
:100ECD00207502D292307502D290206A03020EED87
:100EDD00900298206C0A306E07D2917401D5E0FD16
:100EED00207502C290307502C292207503759F2144
:100EFD00307503759F01753D04D2AF22C2AF206AD4
:100F0D0003020F2B900257306E17207502D29230CC
:100F1D007502D290D2917401D5E0FD020F2E900191
:100F2D00C8C294305A0EE525600A207502D295305C
:100F3D007502D293759F11753D05D2AF22C2AF20B8
:100F4D007502D290307502D292206A03020F74900E
:100F5D000206206C12306E0F207502D2923075028F
:100F6D00D2907401D5E0FDC291207503759F0130BB
:100F7D007503759F21753D06D2AF22C2AF206A035E
:100F8D00020FB290036B306E1F207502D292307536
:100F9D0002D290207502D290307502D2927401D592
:100FAD00E0FD020FB59001EC207502C2953075027F
:100FBD00C293305A0EE525600A207502D293307522
:100FCD0002D295207503759F21307503759F0175AC
:100FDD003D01D2AF229001C6C295C294C293D29266
:100FED00D291D29022C3E54F9535E55095365001FB
:100FFD00227890E6FFC3EF94055018C3EF94045088
:10100D001BC3EF9403501EC3EF94025021C3EF9402
:10101D00015024C3E54F943CF802104DC3E54F94A5
:10102D0028F802104DC3E54F941AF802104DC3E590
:10103D004F9412F802104DC3E54F940AF802104D6B
:10104D00E5509400F9884F8950223058030210570B
:10105D002278847603788576047886760A788F767A
:0F106D0003789076057895760278927603789BD3
:10107C00760D7893760578877603789C7601788858
:10108C0076017889760178827604788C7601788D71
:10109C007600788E76B478967625789776D0789890
:1010AC007678789976C8789A7604789D7600227846
:1010BC0093E6FF756409756501C3BF020975640584
:1010CC00756501021100C3BF0309756405756502DE
:1010DC00021100C3BF040975640575650302110094
:1010EC00C3BF0506756409756507C3BF060675643D
:1010FC00007565007887E6FFC26CC3BF0302D26C33
:10110C00C26BC3BF0402D26BC26A7418552D600245
:10111C00D26AC26E6002D26ED26F6002C26FC275AA
:10112C007888E630E102D275C2767889E630E10241
:10113C00D276C3EF94026008758E01D26D02115104
:10114C00758E00C26D227880E61490008093789E94
:10115C00F67881E61490008093789FF6120FE222C5
:10116C00789BE61490008D9378A0F6120FE222780B
:10117C0086E61490009A9378A1F6120FE222789CDE
:10118C00E6149000A79378A2F6789CE6149000AC35
:10119C009378A3F6120FE222227896E6FA7897E675
:1011AC00FB3077047A007BFFC3EB9AFCC39482502C
:1011BC00027C82756C00056CEC856CF0A4C3E5F0C8
:1011CC00948040F222C2D353D9BF7581C043FF80B3
:1011DC0012073E75EF0243B203E5B324044002F557
:1011EC00B37580FF75A40075F19075D47F759087E9
:1011FC0075A5BF75F2BF75D50075A60175E24112D4
:10120C000FE2E4F8F6D8FD115E12175311BB315200
:10121C00316C317B318A31A431A57898866D120FEF
:10122C00E275885075890275C82475910475D8408B
:10123C0012075212076112074A12076812074A1264
:10124C00076F12074A121CCD1207521207521207CF
:10125C004E75A82275B80275E69075F610759B80D0
:10126C00759D0375D10E75BC5875BB0675BA117595
:10127C00E88012073ED2AF120A5043DA01C2D8C23C
:10128C0069120752753001D2597A05E55770027A06
:10129C0005120742E558C3940240EEE52E541F8513
:1012AC005A59F55AB559E2DAE2C25953DACF2076D7
:1012BC000343DA2030760343DA10C2D8C26912072E
:1012CC004E1207427802741F552E70027800C3E547
:1012DC00589840EDC2AF120761120761120761D234
:1012EC00AF120752754700120742788CE6C394017F
:1012FC0050030213BCE530C3940150030213BC74B9
:10130C001F552E6035C3E55894FF50030213BCC221
:10131C00AF120776D2AF12074EC3E558940150EFC7
:10132C00C2AF120761120746120761D2AF12074E05
:10133C00C3E55894FF40E9021D527F05D27731A5D1
:10134C0012074EC2AFC27731A5C3E558947FD2AF16
:10135C004068C2AF120776D2AFDFE1C3E5589405FF
:10136C007897F61207521217EF121CD57F0AD27714
:10137C0031A512074EC2AFC27731A5C3E558947F91
:10138C00D2AF50E8C2AF120761120746120761D202
:10139C00AFDFDBE55824057896F61207521217EFEB
:1013AC00121D0412074EC3E55894FF40F6021D525D
:1013BC00C3E5589547400385584712074EC3E55877
:1013CC009401400241F3C2AF12077612077612075E
:1013DC0076D2AF120752753000E4F531F532053193
:1013EC00E531F470360532789AE678281460127874
:1013FC005014600D78A014600878F01460037532F6
:10140C0000C3E53298401415327899866DC2AF123C
:10141C000776D2AF7898866D12074E120742E528F0
:10142C007008741F552E70024193C3E55894064002
:10143C00AD12074EE5287003021293120FE2E4F589
:10144C0022F523F524F525755CFF7885865FF53F3D
:10145C00F540F541F542F543F56AF548F52BF52CC9
:0E146C00F55B120B8E756A0875BB1012073EF9
:10147A00120AE8E5E820ECFBA8BDA9BEE97001F86C
:10148A00886B120AEC756A0875BB107895E630E02D
:10149A00030214DA7887E6FE760211BB7887EEF645
:1014AA00D261C2AF120B5E85225C85225DD2AFC2C9
:1014BA0061752500756200756301D260D263753863
:1014CA0000120F4A120F88120C0A120B8E0216090A
:1014DA007887E6FE76037893E6FD760511BB788772
:1014EA00EEF67893EDF6D260D261D26E120F4A12FE
:1014FA000F88120B5E12073E120E4C12073E12079D
:10150A003E120E81120742120ECB120742120742F6
:10151A00120F09120746120F4A12074212073EC259
:10152A0061D262120AE8120AEC120B5E756A087539
:10153A00BB10120F88120C03120C7E120FF21157F5
:10154A00120E4C120C03120C7E120FF21157120ECD
:10155A0081120C03120C7E120FF21157120ECB12CB
:10156A000C03120C7E120FF21157120F09120C0300
:10157A00120C7E120FF21157120F4A120C03120CA0
:10158A007E120FF2C3E54F9535E5509536400C11A2
:10159A0057C3E5589401508B0217231157C262783A
:1015AA0087E6FE760211BB7887EEF685225C855EB9
:1015BA005D855E25756200756301D263753800C268
:1015CA00AF207502D292307502D290207502D29065
:1015DA00307502D292742DD5E0FDD2AF120F881267
:1015EA000C0A120C65120C7E120D02756A0075BB8C
:1015FA000602160911BB120F88756A0075BB06121E
:10160A000D24120DA9120DD1120860120DE5120E49
:10161A004C120C0A120C65120C7E120D02120D1BD2
:10162A00120DA9120DD11208ED120DE5120E81123A
:10163A000C0A120C65120C7E120D02120D24120DE8
:10164A00A9120DD112092D120DE5120ECB120C0A98
:10165A00120C65120C7E120D02120D1B120DA9122C
:10166A000DD112098A120DE5120F09120C0A120C79
:10167A0065120C7E120D02120D24120DA9120DD143
:10168A001209EE120DE5120F4A120C0A120C65121B
:10169A000C7E120D02120D1B120AE8120DA9120D70
:1016AA00D1120AEC120DE5120F88120C0A120C65FF
:1016BA00120C7E120D0230632A755CFF755DFF7590
:1016CA006200756301C3E5389464400AC263D26458
:1016DA007537140216EDC3E5589401400302160942
:1016EA00021723306419E537147005C2640215FE27
:1016FA00F537C3E55894014003021609021723C3BC
:10170A00E55B94825013741F552E7004E528600916
:10171A00C3E53C94F05002C109120FE27887E6FE55
:10172A00760211BB7887EEF6E4F522F523F524F567
:10173A0025F55FC26012073E120FE2741F552E7024
:10174A0006E5287002419361E5901A0D7820121C73
:10175A0000E520B45A0CA3121C00E520B4A503022C
:10176A001774115E1217EF0217EE78827604901A38
:10177A00077884121C00A308121C00A308121C007C
:10178A00A308121C00A308121C00A308121C00A321
:10179A0008A308A308121C00A308A308A308121C84
:1017AA0000A308121C00A308A308121C00A3081215
:1017BA001C00A308A308121C00A308121C00A308FB
:1017CA00121C00A308121C00A308121C00A3081272
:1017DA001C00A308121C00A308121C00A308121C58
:1017EA0000901A2122C2AF121C3F121C19901A0033
:1017FA00740A121C05A37404121C05A37410121C8B
:10180A0005901A077884121C04A308121C04A30862
:10181A00121C04A308121C04A308121C04A3081215
:10182A001C04A308A308A308121C04A308A308A362
:10183A0008121C04A308121C04A308A308121C04FF
:10184A00A308121C04A308A308121C04A308121C50
:10185A0004A308121C04A308121C04A308121C04E3
:0F186A00A308121C04A308121C04A308121C04D8
:0F187900A308121C04121C52121C30901A2122B8
:101A00000A0410FFFFFFFF03040A0301015AA501A6
:101A1000FFFF0305FF0305FF0225D0FAFA040D01BD
:021A200000FFC5
:101A400023585032354123202020202020202020E0
:101A500023424C48454C4923463333302320202031
:101A60002020202020202020202020202020202076
:101C0000E493F622E6438F01538FFD75EF0275B71B
:101C1000A575B7F1F0538FFE22438F02438F0175F4
:101C2000EF0275B7A575B7F1901A0DF0538FFC222E
:101C3000901A0D745A9105901A0E74A59105227A86
:101C40003079D07820901A409100E520F709A3DA86
:101C5000F7227A3079D0901A40E7910509A3DAF992
:101C600022AB6EA86FBB01057984021CCABB0205BA
:101C70007985021CCABB03057995021CCABB040501
:101C80007986021CCABB0505798F021CCABB0605F2
:101C90007990021CCABB07057992021CCABB0805D1
:101CA000799B021CCABB09057993021CCABB0A05B1
:101CB0007987021CCABB0B05799C021CCABB0C05A8
:101CC0007988021CCA7989021CCAE8F7227C0512AD
:101CD0000752DCFB22C2AF12076112076812076FBE
:101CE00012077612074612076112076812076F1271
:101CF000077612074612076112076812076F12076C
:101D000076D2AF22C2AF12077612076F120768129F
:101D1000076112074612077612076F12076812074B
:101D20006112074612077612076F120768120761E1
:101D3000D2AF22AE6EAF6FC2AF120761120761124F
:101D40000761120746DEF2120776120746DFF8D265
:101D5000AF2291D591CD91CD756E01756F017570E2
:101D600000B1337C05AD58120752C3ED955870F59C
:101D7000C3E55894014009C3E55894FF4032A18E51
:101D800091611217EF91D5C2AF75EF1291CDDCD5ED
:101D90000570C3E5709403500280C691CD056FE5D0
:101DA0006E149000B193F808C3E56F98500280AEAE
:101DB00091CD91CD056EC3E56E940E5002809C12BC
:0C1DC000105E1217EFC2AF75EF1291CD4C
:00000001FF
